:020000040000FA
:040000006F303A28FB
:08000800A000030EA100831209
:100010008B1C32288B1031181428B11C3228643004
:10002000010203183128182800001628172818285C
:1000300019281A281B281C281D281E281F283110A3
:10004000B114A810031005190314AA0DA90DA80DC9
:10005000B00B322831152A08AF002908AE00280855
:10006000AD00B11081010B11210E8300A00E200EF6
:02007000090085
:0C007400203084008001840A80300402E7
:10008000031C3C281230B0006B2183160C30850510
:1000900087018312850187010730990000309A009B
:1000A000103083168E008312603083168F00831207
:1000B0000030831691009F008312C83083168100A0
:1000C000831231309000003083168C008312103080
:1000D0008B00A92181018E018F010B118B100B1058
:1000E0008C018B178220311998204D21B30B802869
:1000F000031085190314B90DF03039020319F620E5
:10010000AA2172286400311808000B1D08000B1189
:10011000B11031141230B000051D9328321483162B
:10012000011383120800321083160117831208008E
:1001300031110130B7008B132030370783169B0035
:100140001C141A088312A400A500C030A5061030A4
:10015000370783169B001C141A088312A300003073
:10016000370783169B001C141A088312A2008B17F2
:10017000321CC02822090339A200A309A409A50939
:1001800022082D02031DF02823082E02031DF0284B
:1001900024082F02031DF02801303702031DD52843
:1001A0003D18D5283D143E14862102303702031D28
:1001B000DE28BD18DE28BD143E148F21033037021F
:1001C000031DE7283D19E7283D153E14982104300A
:1001D0003702031DF028BD19F028BD153E14A121DA
:1001E000B70A05303702031808009B280130B60013
:1001F000B300B400B500B70085018701B1138220B8
:10020000B30B1C29031085190314B90DF030390202
:1002100003194329B41F8501B41F8701B40B1C299E
:100220003708B6080319B60003191A29FF308500EC
:100230008700B6039630B400311DFF283111321CFF
:1002400026292D090339AD00AE09AF092F1CB113C2
:100250002F1CFF28B11BFF282E18FF28B1178B1366
:1002600020303707BB002F08BA005621103037075F
:10027000BB002E08BA00562100303707BB002D08FE
:10028000BA0056218B1785018701B70AB6010530E0
:100290003702031CFF28A92108003E1C08003E105D
:1002A0001030BB003D08BA00562108008B133A08F5
:1002B00083161C159A0083123B0883169B00553049
:1002C0009D00AA309D009C1464009C1864291C1198
:1002D00083128B170800831610309B001C141A0819
:1002E0008312BD00831620309B001C141A08831251
:1002F000C2000130C21BC200C2080319C200013093
:10030000D500D200EE30D000D10008000130D50079
:10031000D200EE30D000D1000130BD000800013025
:10032000D500D200EE30D000D1000230BD00080070
:100330000130D500D200EE30D000D1000430BD0035
:1003400008000130D500D200EE30D000D100BD0150
:10035000080008008F08031908008F01C10B08006E
:100360004208C100D50B08005608D50007303D05EE
:100370000319E129D21BD00AD21FD0030A30500240
:10038000031CDC29D0010930D21FD0005203D20057
:100390007F39031DDC29D10A10305102031CD129F9
:1003A000D1015022D2006022D4007022D600D500A4
:1003B000D0010930D21FD0000023850024238700FC
:0803C000080085018701080017
:1004A00002308A0051083D1C572A883E8200BD1C3C
:1004B0005B2A883E82003D1D5F2A983E8200003400
:1004C00002308A0051083D1C672AA83E8200BD1CEC
:1004D0006B2AB83E82003D1D6F2AB83E8200003470
:1004E00002308A0051083D1C772AC83E8200BD1C9C
:1004F0007B2AD83E82003D1D7F2AE83E82000134DF
:100510000734873407348734033483340334833413
:100520000B3403340F3407340B34033403340734EF
:10053000053487340734253483340334073489344D
:100540000B3403348F3405348B34113403340334C7
:1005500001340134023402340434043408340834DD
:10056000103410342034203440344034803480340B
:10057000083404340234803440348034103402347B
:10058000043410342034013404344034843480344E
:10059000093409340A340A34083408340834083475
:1005A0000834183408341834083418341034083433
:1005B000093429340A341A34283408340834083405
:1005C0000A34383408341A3408345834103448346F
:1005D000293409340A340A342834083408344834B5
:1005E0002834183488341834283418341034083433
:1006000003308A005008541C072B4B3E8200D41C38
:100610000B2B563E8200541D0F2B613E8200D41DD1
:10062000132B6C3E8200541E172B773E8200D41E83
:100630001B2B823E8200541F1F2B8D3E8200D41F35
:10064000232B983E8200003403308A005008541C4B
:100650002B2BA33E8200D41C2F2BAE3E8200541DB8
:10066000332BB93E8200D41D372BC43E8200541E6A
:100670003B2BCF3E8200D41E3F2BDA3E8200541F1C
:10068000432BE53E8200D41F472BF03E820000340E
:0A0696001034203401340234003423
:0A06A000003400340034003400344C
:0406AC0010343034A2
:1006B0003134333433343334333433343334333404
:0E06C2000034003400340034003400340234BC
:0606D0000334233433342F
:0806D800103420340134023417
:0C06E000003410342034013402340034A3
:0206EE001034C6
:1006F0002034013402340034003402340134203414
:020700001034B3
:0C070400103430343134333433343334A7
:080710003134303410340034A0
:06071A00333423340334E4
:0E072000023400340034023403342334333402
:10073000333400343334003433340034333400344D
:04074000333400341A
:0A07460000340034003400340234A3
:0A075000043401342034103408345E
:04075C000034003431
:1007600000340034023406340734273437343F343D
:0E07720008341834383439343D343F343F34C1
:060780003F343F343F341A
:08078800043401342034103464
:0C0790000A3404340134203410340A34DC
:02079E0008341D
:1007A000103420340134063406340134203410343B
:0207B00008340B
:0C07B40008341834383439343F343934F8
:0807C000383418340834003409
:0607CA003F3437342734F0
:0E07D0000734063406340734273437343F34F8
:1007E0003F3400343F3400343F3400343F3400346D
:0407F0003F3400345E
:084000000C000300060006009D
:02400E00CC33B1
:10420000010003000300030003000200020002009B
:1042100002000000000000000000FF00FF00FF009F
:10422000000000000000000000000000000000008E
:104230000000C000C000C000C000FF00FF00FF0081
:104240000100C300F300CF00FF00C300F300CF0064
:10425000FF00C300F300CF00FF00FF00FF00FF00DE
:10426000FF00FF00FF00FF00FF00FF00FF00FF0056
:10427000FF00FF00FF00FF00FF00FF00FF00FF0046
:10428000FF00FF00FF00FF00FF00FF00FF00FF0036
:10429000FF00FF00FF00FF00FF00FF00FF00FF0026
:1042A000FF00FF00FF00FF00FF00FF00FF00FF0016
:1042B000FF00FF00FF00FF00FF00FF00FF00FF0006
:1042C000FF00FF00FF00FF00FF00FF00FF00FF00F6
:1042D000FF00FF00FF00FF00FF00FF00FF00FF00E6
:1042E000FF00FF00FF00FF00FF00FF00FF00FF00D6
:1042F000FF00FF00FF00FF00FF00FF00FF00AA001B
:00000001FF
